:060000000207D402191EE4
:03000B0002184692
:03001300021A745A
:1000230002276000000E010F110F0200000E111FC6
:10003300100E0202040E1010110E0018080C0818FE
:10004300081C00020416191111110002040E1111EB
:10005300110E0002040E100E011E0006001F020402
:10006300081F00C287749612010174301200B7741E
:100073003212010174301200B7740212010174309C
:100083001200B7742844301200C674081200C674F4
:10009300011200C674061200C6740F1200C6744023
:1000A3001200C67A40900026E4931200D5A3DAF832
:1000B30012018F22120151C286C285D287C287D212
:1000C30085C3221200E4500122C286C285120114A4
:1000D30080E91200E4500122D286C2851201148005
:1000E300DAC0E0D2A7C286D285D287740030A708CF
:1000F3000000D5E0F8D38001C3C287D0E022C0E07E
:10010300C0F0F5F07460D5E0FDD5F0F8D0F0D0E0A4
:1001130022C0E0C2A0C2A1C2A2C2A3C2A4C2A5C2FD
:10012300A6C2A730E002D2A030E102D2A130E2029F
:10013300D2A230E302D2A330E402D2A430E502D249
:10014300A530E602D2A630E702D2A7D0E022C0E073
:10015300C2A4C2A5C2A6C2A780DDC0E0740C12006F
:10016300C6D0E022C0E0740D1200C6D0E022C0E089
:1001730074021200C6757F00D0E022F57FD2E70239
:1001830000C6C394082440D2E70200C6C0E074014D
:100193001200C6757F00D0E022E5831201AC40084F
:1001A300E5821201AC4001C322C0E0C0F0C082C0AE
:1001B30083F5F003030303540F90023893120704EB
:1001C300400EE5F0540F900238931207044001C328
:1001D300D083D082D0F0D0E022C0F075F00833C0D5
:1001E300E0743050027431120704D0E0D5F0EFD040
:1001F300F022C0E003030303120201D0E022C0E0B7
:10020300C082C083540F900238931207044001C385
:10021300D083D082D0E022C082C083C0E003030336
:1002230003540F90023893F8D0E0540F90023893A0
:10023300D083D082223031323334353637383941A6
:100243004243444546B40C0302018FB40D0122B46A
:100253000A0302029CB4FD03020171C0E0C0F085F1
:100263007FF0C0E07410B5F00612029C857FF0D0D9
:10027300E0C0E0E5F0D2E71200C6D0E01200D5807E
:1002830011E5F0C394082440D2E71200C6D0E0126F
:1002930000D5057FD0F0D0E022C0E0744012017E8B
:1002A300D0E022C0F0C082C083E493602DB4FB137E
:1002B300A3E493F5F0A3E493120704401AD5F0F8EE
:1002C300A380E6B4FA09A3E49312017EA380DA12B1
:1002D30007044003A380D2D38001C3D083D082D04C
:1002E300F022C0E07420120704D0E022C0E0740DB5
:1002F300120704D0E022C0E0740A120704D0E022FF
:10030300C0E0740D1207044008740A120704400188
:10031300C3D0E02275F06484C0E0E5F075F00A8490
:10032300C445F0D0F022B441004007B45B00500252
:10033300D2E522B461004007B47B005002C2E5223B
:10034300B461004008B47B005003C2E522B441000D
:100353004007B45B005002D2E522C0F08FF0C0F03A
:10036300D2E0F5F07F001203AAE5F01203D2400EAB
:100373001204081203C2C3D0F0AFF0D0F02212036C
:10038300C27401120436DFDED380ECC0F075F000D6
:100393001203C2500AD284D283C283D5F0F2D3D0DF
:1003A300F0C27522207512D283D28430830B30843D
:1003B30008C284C283C3D27522D3D283D28422C219
:1003C30084D283D2843083F13084EEC3C27522C0D9
:1003D300E0C0F075F008334004C2848002D2841276
:1003E300041A120414D5F0EED28412041AA2841251
:1003F3000414D0F0D0E022120420C28412041A1292
:100403000414D28422120420D28412041A12041473
:10041300223083FDC28322D2833083FD22C0F07554
:10042300F008D28412041AA28433120414D5F0F40F
:10043300D0F022C0E0C0F0F5F07460D5E0FDD5F057
:10044300F8D0F0D0E0227A0478337937E6C3977096
:100453000D1819DAF7C27EC27DD27C0204724009FC
:10046300C27CC27DD27E020472C27CC27ED27D2255
:100473007F0A7E0078409004FF7A04793877000978
:10048300DAFB7938E66020FDEE2323FBEBFC9327B0
:10049300F70C09EC9337F70C09EC9337F70C09ECDD
:1004A3009337F77938DDE5080EDFD9227838794AB2
:1004B3009005277E007A05770009DAFB794A7D04E7
:1004C300E6FC7B08EC13FC501875F005EEA4FA7FEC
:1004D30005C3EA937002500737D4F70A09DFF379AB
:1004E3004A0EDBE008DDD9794A78407F05E7540FEF
:1004F300F608E7C4540FF60809DFF22201000000F2
:100503000A00000064000000E80300001027000058
:10051300A086010040420F008096980000E1F50597
:1005230000CA9A3B01000000000200000000040022
:100533000000000800000000160000000032000068
:1005430000006400000000280100000056020000C3
:1005530000120500000024100000004820000000E5
:10056300964000000092810000008463010000684F
:1005730027030000365506000072101300004421C3
:10058300260000884252000076850401005271095A
:10059300020004431904000886380800167277160F
:1005A30000324455330064881067002877213401F2
:1005B3005654436802120987360524187473104889
:1005C300364847217F0479387A307B34C3EAF8E62A
:1005D300FCEBF8EC36F7090A0BDFF2227F047938DB
:1005E3007A307B34C3EAF8E6FCEBF8EC96F7090AB9
:1005F3000BDFF2500B7F047938770009DFFBD27FE2
:100603002278387F04760008DFFB7834794A7F0448
:10061300E6F70809DFFA7B307C02EBF8E6FA7F089D
:10062300C3EA13FA500E7838794A7E04C3E637F6E4
:100633000809DEF9C37E04784AE633F608DEFADFFA
:10064300DF0BDCD62278377F047B20E67E0833403D
:100653000E1BDEFA18DFF4EB7005D27F0207037876
:10066300337F047C20E67E083340061CDEFA18DF65
:10067300F4C3EC9B4075FAFB0B7830794A7F04E6B0
:10068300F70809DFFAEA600DC37F047834E633F62E
:1006930008DFFADAF37F047838760008DFFB7F049B
:1006A300C37838E633F608DFFAC37F04784A79342F
:1006B300E6970809DFFA4011C37F04784A7934E6E4
:1006C30097F60809DFF9783806EBC39401600B7FCE
:1006D300047837C3E613F618DFFADBC2784A793CAD
:1006E3007F04E6F70809DFFA0207037830793C7FD5
:1006F30004E6F70809DFFA78387F04760008DFFBA1
:1007030022C0E0E550B4030AD0E0C0E0120729D0CC
:10071300E022B4020AD0E0C0E01207AED0E022D05B
:10072300E0120248C32285115112269DC0E0E50F55
:10073300B40207D0E01207C9C322D0E01207514028
:100743000B12076DC2810000D281C322D322C0E005
:10075300751F0A122EE8208004C3D0E022120EEC8B
:100763004004E51F70EDD3D0E022C0E0C2A7C2A6CB
:10077300C2A5C2A4C2A3C2A2C2A1C2A030E002D237
:10078300A730E102D2A630E202D2A530E302D2A41E
:1007930030E402D2A330E502D2A230E602D2A13085
:1007A300E702D2A0D0E02275170022851251B40CC3
:1007B3000A740A1207C9740D0207C9B4FD0122B4F1
:1007C300FC012212269D3077FDF599122EE8C2779F
:1007D3002275818078BF765418E8B480F91207AA8D
:1007E300121A5A12182C122805122824122812122F
:1007F300281B12184312006612038E122EF2120ADD
:100803001312018F1217CF122ECE1228E7121FAE2A
:1008130012015D1216EC20950312348212337575A2
:1008230016001228C0E517B40002C282D295755093
:1008330001121F5012281B12015D122AD89008D4EE
:100843001202A61214271202E51202E512298312DC
:1008530009E5209205D282120DFF1215BD404130E9
:10086300D5C0D2829009B81202A6120A49120BC54A
:1008730078321228A61215BD400720D5F3D8F3010C
:100883001F30760C7828E50E30E0151228A6D8F62E
:100893009009C31202A6120BC51215BD40FB011F1E
:1008A300D28212169BC27A121FBB1216049009CE73
:1008B3001202A612016778F012160E500302081FE7
:1008C300B40E028020B8FE0280EEF61226270880BE
:1008D300E7FD0D0A2020202020202020202020209A
:1008E300202020200012015D12018FE5F0B4FF03E8
:1008F30002081F9009D41202A6121FBB121FA512D1
:1009030014E0121E95121B4B740A12289B1216E94F
:1009130012015D122EE8120171740112289B121349
:10092300C61213691228B33090E93091E61228B346
:100933003090E03091DD120D59120D6F120C64D21C
:10094300E7120D33120D8F751500E561120D33E5B6
:1009530062120D33E563120D33E564120D337F0626
:1009630078F0E62323232354F0F5F008E645F0124C
:100973000D3308DFEDE574120D33E575120D33E524
:1009830076120D33E577F518120D33E578F5191264
:100993000D33E515120D33740A12289B75F0C81236
:1009A30015BD500302081F740112289B122AD8D5C3
:1009B300F0ED02081F0C447A776F6E656B2E2E00E4
:1009C3000C526F7A6D6F77612E2E000C4E723A20A7
:1009D300000C4F6B7265066C616D207461727966F1
:1009E3000100307B2A78F0121678757E06122EE805
:1009F300307B0A1216782430757E06F60830930889
:100A0300E57E70E975160022E8C394F014F516220A
:100A1300C2A9C2A81203AA74401203D274FB120320
:100A2300D21203C2D2A9D2A8C29622C2A9C2A812C4
:100A330003AA74401203D274F71203D21203C2D270
:100A4300A9D2A8C2962275F005122EE81228C0304A
:100A530093F4D5F0F4755002120A2E1228A6122828
:100A6300A6C278120B724012120B72400D120B7257
:100A73004008120B724003020AE4900C2C1202A6E7
:100A8300120B72505DB455F8120B725055B480F8C6
:100A93007D80120B72505B120704FF120B725052CF
:100AA300120704FC1F120B725048120704FE1F1298
:100AB3000B38503EEFB400E3C374009DF5F0120B06
:100AC30072502F120704B5F038120B21854161854E
:100AD3004362854563854764121AB5755001120A4E
:100AE3001322122D54900AF01202A680EE53594E8F
:100AF3004300122D54900B001202A680DE42524B8B
:100B030000122D54900B1B1202A6C0E0E5F0120157
:100B1300ACD0E01201AC80C34352432024007840A0
:100B23007F04E6C39430F5F008E6C39430120EDB7D
:100B3300F608DFEE22ECB402138E1678F0120B7275
:100B4300502C120704F6081FDEF3D322B401138ED0
:100B5300167840120B725016120704F6081FDEF3C4
:100B6300D322120B7250071207041FDEF5D322C0E3
:100B7300F075F000122EE8120BA930E40A1228D8FF
:100B8300D5F0F1D0F0C322D0F0C278C0F075F008F0
:100B9300A29713D2960000C296D5F0F4C0E02DFDC3
:100BA300D0E0D3D0F022C2A9C2A81203AA74401283
:100BB30003D21203AA74411203D2120408D2A8D298
:100BC300A922C050755001120BE2755002900C3DE2
:100BD3001202A61214271202E5120BE2D05022E5EC
:100BE300166032E550B4010312030378F0AF16E642
:100BF300B4300908DFF9900C190202A6B450028040
:100C0300F5B44F06900C200202A6AF1678F0E61258
:100C1300070408DFF922416E6F6E696D004E696546
:100C2300646F737401706E79000D0A2346534B2071
:100C3300000D0A2344544D4620000D0A23436C69DA
:100C4300703A2000C083C082120C64C0D0855782E2
:100C5300855683A3858257858356D0D0D082D0838F
:100C630022C083C082855782855683120C83C0E0DD
:100C7300122AACD0E0D082D08330E702D322C32241
:100C8300122EE8C0F0C083C082C2A9C2A8120D22EE
:100C93001203AA74A045F01203D24027E58312037E
:100CA300D2E5821203D21203AA74A145F01203D231
:100CB30040111204081203C2D2A9D2A8D082D08351
:100CC300D0F022755001122D54900CD51202A602B9
:100CD3002EA7454570726F6D00122EE8C0F0C083D9
:100CE300C082C0E0C2A9C2A8120D221203AA74A036
:100CF30045F01203D240CCE5831203D2E5821203FE
:100D0300D2D0E0C0E01203D21203C274A145F012A4
:100D1300035DD2A9D2A8D0E0D082D083D0F022E55F
:100D23008303030303540EF5F0E583541FF5832275
:100D3300C0E0C083C082C0F0F5F08557828556833A
:100D4300120CDC122AACA3858257858356D0F0D0CF
:100D530082D083D0E022120D67120C644005120D7D
:100D63006F80F6227525007526008045E525B52799
:100D73000AE526B52805120D67D322E5252401F5DA
:100D830025E5263400F526120DB4C322E525700FA0
:100D9300E526700B852725852826120DB4D322C39B
:100DA300E5259401F525E5269400F526120DB4C337
:100DB30022C083C082852582852683E58233F5821E
:100DC300E58333F583E58233F582E58333F583E504
:100DD3008233F582E58333F583E5823354F0F5827C
:100DE300E58333F583E5822420F582E583340EF52C
:100DF30083858257858356D082D0832212015D1268
:100E0300117675100312015D1215BD40143092F571
:100E1300900F4C1202A61215BD40153092F8D295D0
:100E230022C295740112289B1232F420D5E240F1BC
:100E330012015D7900120E6740F6120F0B20D5D018
:100E430050030980F012018F120167F5F012262773
:100E5300120F0B20D5BA40D8122627120EDB121020
:100E630071020E33E9B41002D322E92354FEF5F0E4
:100E730090105193FFE5F00490105193F5838F8206
:100E830012015D1202A6C322C2D18010C2D1C0F0EA
:100E9300E57F12017E75F000802AD2D1C0F0E57F94
:100EA30012017E120F0B20D52C40F8B40A00400C1F
:100EB300F5F02323232354F045F08019F5F020D1D6
:100EC30003122627120F0B20D50B40F820D1031253
:100ED3002627120EDBD0F022C0E0E5F023232323E4
:100EE30054F0F5F0D0E045F022C0E0E510B4020A7A
:100EF3001227A8500FB41B0C8006309007309104C2
:100F0300D0E0D322D0E0C322122EE8E550B4020F82
:100F130012283D4030B41B02801BC39430801A1248
:100F23001FBB757E023090053091028003307B0D2C
:100F330012160E5004D2D5D322C2D5C322122EE8E4
:100F4300E57EB400E0C2D5D3220C2A2A20577903C8
:100F530008637A2050524F47202A000C31312D4C20
:100F630069637A6E696B69000C37312D4472756B56
:100F7300206275666F7261000C37322D4472756B97
:100F83002070726566696B73000C37332D4472757C
:100F93006B207461727966000C37342D4472756B63
:100FA300206B6F6E666967000C37392D4472756B61
:100FB30020706F20434C52000C39312D55737461EE
:100FC300772070726566696B73000C39322D557327
:100FD30074617720746172796679000C39332D431B
:100FE300656E61000C39342D437A6173000C393519
:100FF3002D5A616C69637A616E6965000C39362D0F
:101003004472756B61726B61000C39372D537461D7
:101013006E6461726420504C000C39382D4A617340
:101023006E6F0602204C4544000C39392D4B6F641A
:10103300000C30302D5374616E64617264000C30A7
:10104300312D4B6173756A206275666F72005E0F96
:101053006B0F7B0F8C0F9B0FAB0FBB0FCD0FDE0FF7
:10106300E70FF00FFF0F0C102C1034104110B411C8
:1010730005121176C322B47105122186C322B472FC
:1010830005122578C322B473051224B9C322B4749C
:1010930005121FDFC322B47905122182C322B49142
:1010A30005122EF3C322B49205123156C322B49310
:1010B300051212C3C322B49405121236C322B49587
:1010C300051212FCC322B49605121132C322B4973F
:1010D300051210F3C322B4990512331DC322B400C1
:1010E30005123482C322B4010512219EC322D322E6
:1010F30012016790111C1202A6120F0B20D5174084
:10110300F8F5119011261202A6120F0B20D50740F5
:10111300F8F512122A270203030C50727420504C64
:101123003A20000C525332333220504C3A200012F2
:1011330001679011511202A612132520D50D400507
:10114300750F018003750F02122A270203030C5047
:10115300727420302D50617220312D53657200124C
:101163000D67120C64D2E7120D33120D6F50F31298
:1011730007AA2212018F85278285288375F085129D
:101183001781742F1207041211CC8A828B8375F096
:10119300841217811203031211CC75F0881223F500
:1011A300742F120704AD18AC197F007E0075F0850B
:1011B3001223F5122EE83092FA75F0141228A63095
:1011C3009204D5F0F7220233B37C007D007E007FCA
:1011D300007A007B00121211500122120C47402D9D
:1011E30075F00C1224A8120C47C0E0120C472CD443
:1011F300FCD0E03DD4FDEE3400D4FEEF3400D4FF48
:10120300EA2401FAEB3400FB120D6F80CE22120D9B
:1012130059120D6F900000120C645015A3E582B5AE
:10122300270AE583B52805120D67D322120D6F80B7
:10123300E6C3229012B01202A6120167757F001254
:101243000E8B20D567F57B120E8B20D55FF57C7551
:101253007F05120E8B20D554FAB4130050F1B4015C
:101263000040EC757F08120E8B20D540FBB4320092
:1012730050F1B4010040EC9012BC1202A6757F003D
:10128300120E8B20D526FCB4240050EB757F03127D
:101293000E8B20D517FDB45A0050F18C638D648BEF
:1012A300628A61857B66857C65121AB5220C52526F
:1012B3005252204D4D2F4444000C67673A6D6D0028
:1012C3009012EE1202A6120167757F05120E8B2093
:1012D300D514FA757F08120E8B20D50AFB8B5A8A18
:1012E300598C58122A27740A02289B0C43656E6195
:1012F300203F3F2C3F3F7A03009013161202A612A1
:101303000167757F0B120E8B20D505F579122A27FD
:101313000203030C5A616C69637A616E6965203F4D
:101323003F00120F0B20D50740F8B40102D322C3AC
:1013330022C05075500112016790134DE510B4029D
:101343000390135B1202A6D050220C4472756B6F8C
:1013530077616E69652E2E000C4F627303756761AA
:101363002052532E2E00744512017EE55D120201B8
:10137300E55E1201AC742E120704E55F1201AC7432
:101383004012017E7474120704E5671201AC221245
:101393000303855C827583001215261213AE1202B5
:1013A300E57474120704E5670201AC12157278093B
:1013B300120C836008120704A3D8F580051202E516
:1013C300D8FB22E5741201AC743A120704E57512D6
:1013D30001AC743A120704E5761201AC1202E5126D
:1013E30002E5E577FD7F007E00E578FC75F00512E8
:1013F30023F522E5741201AC743A120704E5751261
:1014030001AC743A120704E5761201AC1202E5123C
:1014130002E51202E5744C120704E5771201ACE50C
:10142300780201AC120171121B4BE56012146312B6
:1014330002E5E5621201AC1202E5E56112148512C0
:1014430002E5E5631201ACE550B40109E524B405F6
:101453000074204002743A120704E5641201AC22BE
:101463002354FEF5F09014779312070405F0E5F08A
:10147300930207044E69506F57740672437A50699A
:10148300536FB40F004003C3940614232354FC90FA
:1014930014B02582F582E5833400F583E4931207C3
:1014A30004A3E493120704A3E49302070453747997
:1014B300204C7574204D6172204B7769204D616A11
:1014C30020437A65204C6970205369652057727AEE
:1014D30020506107204C697320477275207E007588
:1014E3005C009000007F0078F07968121526402692
:1014F300E7B40F02800DE6F5F0E7B5F0160F080923
:10150300B974EDBF0002800BEEB507005005AE07BE
:1015130085825CA380CF855C827583001215268546
:10152300675B22C0E0C0F088F0C0F0C082C083AA2D
:10153300827583001215837867120C83B4FF03D37B
:101543008020F608A3120C83C0E003030303540FA7
:10155300F608D0E0B874028008540FF608A3B874F4
:10156300E4C3D083D082D0F0A8F0D0F0D0E022C082
:10157300E0AA82121583A3A3A3A3A3A3A3D0E0226B
:10158300EA33F582740033F583E58233F582E5832C
:1015930033F583E58233F582E58333F583E58233DF
:1015A30054F0F582E58333F583C0E0E58224A0F5AA
:1015B30082E5833401F583D0E022122EE87F0A20EE
:1015C30093071228C0DFF88034309007309104C3AA
:1015D300C2D5227F467E007D001228D83090063087
:1015E30091030E80010DDFF1EDB445004004D3C239
:1015F300D5222076DA80D8EEB4020040D2C3D2D509
:101603002278F0740FF608B8FEFB22C0F08FF0C00A
:10161300F07F01122EE81216AF5004740E803E3094
:101623007B08121678121FBB80333090E63091E3AB
:101633001228C03090DD3091DA74001228D804B437
:101643000003D3802930900530910280EE1228C028
:1016530074001228D804B4000CEF121FBBB40A02A2
:101663007400C380093090EA3091E70F80A5D0F071
:10167300AFF0D0F022E5B075F00030E702D2F030E1
:10168300E602D2F130E502D2F230E402D2F3E5F021
:10169300B40A027400C27B22E5905403F57A22E572
:1016A3009054036403B57A02D322C322E579B400CC
:1016B300071216A2402EC322B40107207A26C27A4B
:1016C300C322B40215E523B40800400CB40C005047
:1016D30007E520B43200500CC322309207B57600E0
:1016E3004002C322D322C27A229017251202A67483
:1016F3001912289B122B999017481202A6743130A5
:10170300760274321207049017551202A69036A17E
:1017130012019C90175B1202A6122B6274191228F5
:101723009B220C52656A6573747261746F72203206
:101733002E33320A28432932303033204279205263
:101743002D4D494B000C48617264776172653A20F4
:1017530056000A526F6D2000205265762E313135C6
:1017630000C0F0121E2AE583121E1B85F043F542CA
:10177300E582121E1B85F041F540D0F08015C0F0C4
:10178300858238858339753A00753B001204AFD0E2
:10179300F08000C2D130F702D2D1E5F0543FF5F02A
:1017A300743F25F0F8D2D5E630D5196004C2D58050
:1017B30013E5F0B40106C2D57430800820D10812B5
:1017C30002E5800312020118D5F0DC2290181C7880
:1017D300001203AAE4931203D240321203C29018F8
:1017E30024E893F51E751DF0C3E51D9420F582E5ED
:1017F3001E940EF58375F004C3E58313F583E58228
:1018030013F582D5F0F2858227858328221203C23D
:10181300A308E8B408BB020CC6AFADABA9A7A5A348
:10182300A1FFDFBF9F7F5F3F1F5389F0438901758E
:101833008CB2758A10757D02752402D28CD2A922CE
:10184300D2AF22C0D0758CB2758A10D26BC0E0C003
:10185300F0C000C001C002C003C004C005C006C080
:1018630007C083C082051CE51C20E002051BD57D53
:1018730039757D0A1218CFD5243075240AE57E60A8
:1018830002157EE51F6002151FE5762401D4F57667
:10189300B46017757600E5752401D4F575B4600A54
:1018A300757500E5742401D4F57400121E491218ED
:1018B300FFD082D083D007D006D005D004D003D088
:1018C30002D001D000D0F0D0E0D0D032E50E30E02D
:1018D30015E52060020520E521B40102801D852164
:1018E300237521018015E52160020521E520B4015E
:1018F300028008852022752001800022C00078BF65
:10190300E6B45403D00022755001122D54901919D6
:101913001202A6022EA753746F7300C082C083C045
:1019230007C006C005C004C003C002C001C000C098
:10193300F0C0E0C0D0207604D27A80291203AA74C2
:10194300401203D21203AA74411203D2120408C034
:101953000EF50ED02A1203C2E50E20E602802112F4
:101963001A34121A47D0D0D0E0D0F0D000D001D032
:1019730002D003D004D005D006D007D083D0823262
:10198300755002D2AFD2ACD2BCD277C29912030344
:101993001203031214279019FC1202A6D0E01201BD
:1019A300AC1202E5D0E01201AC1202E5D0E0120164
:1019B300AC1202E575F008D0E01201AC1202E51298
:1019C3002EE8D5F0F2D0E01201ACD0E01201AC1257
:1019D30002E5D0E01201ACD0E01201AC1202E5D076
:1019E300E01201ACD0E01201AC1202E5D0E012012A
:1019F300ACD0E01201AC022EA70D0A5053204120B7
:101A030020422020523020523120523220523320A3
:101A1300523420523520523620523720647074726B
:101A230020504320202050433220205043330D0ABE
:101A330000E50E652A5402B40209E52A5402B402F1
:101A430002D27A22E50E652A5410B41009E52A540D
:101A530010B41002D27822C274C273751A007508CA
:101A630000750900750A00750B00750C00750D00F3
:101A730022C0D0D27BD0D032C007C083C082FFE562
:101A8300F0901AA5934FD082D083D00722C007C00D
:101A930083C082FFE5F0901AAD935FD082D083D0EC
:101AA30007220102040810204080FEFDFBF7EFDF50
:101AB300BF7FC2A9C2A81203AA74D01203D2407373
:101AC30074201203D2406C1203C21203AA74D01200
:101AD30003D2405F74001203D24058E5631203D26D
:101AE3004051E5641203D2404AE5621203D24043F7
:101AF300E5611203D2403C1203C2D2A9D2A8021B51
:101B030004C2A9C2A81203AA74D01203D240247437
:101B1300041203D2401DE5661203D24016E5651296
:101B230003D2400FE5F01203D240081203C2D2A938
:101B3300D2A822755001122D54901B451202A60201
:101B43002EA75A6567617200C2A9C2A81203AA74BC
:101B5300D01203D240DD74001203D21203AA74D14F
:101B63001203D240CE1203FAF5631203FAF564129C
:101B730003FAF562120408F5611203C2D2A9D2A8CE
:101B8300121B95121C72121BC9121C3E021C1C0252
:101B93001B36C2A9C2A81203AA74D01203D240935F
:101BA30074041203D21203AA74D11203D240841212
:101BB30003FAF5661203FAF565120408F5F0120349
:101BC300C2D2A9D2A822121B95E561B4122AE562FA
:101BD300B43125D2F1C2A9C2A81203AA74D0120348
:101BE300D240AC74061203D240A5E5F01203D240F2
:101BF3009E1203C2D2A9D2A8E561B4011BE562B467
:101C0300011630F113E5652401D4F565E56634006A
:101C1300D4F566C2F1121B0422121B95E561B403CD
:101C230019E562B4250050028010E560B4000BE5AD
:101C330063B40206756303121AB522121B95E5619C
:101C4300B4102BE562B42405D2F2121B04E562B48E
:101C5300250050028018E560B40013E563B4030E59
:101C630030F20BC2F2121B04756302121AB5221270
:101C73001E2AE566121E1B85F043F542E565121E1A
:101C83001B85F041F540120473783879E4121E0C79
:101C9300121E2AE561121E1B85F041F540120473E2
:101CA300783879EC121E0C121E2AE562121E1B856F
:101CB300F041F540120473783879E8121E0CE5619F
:101CC300B403004002801078E475F001121DF77828
:101CD300EC75F00C121DE378E479DC121E0C78E449
:101CE3007930121E0C75340475350075360075375E
:101CF30000120648783879E0121E0C121DB378E4FE
:101D03007930121E0C7534647535007536007537DD
:101D130000120648783879E0121E0C121DCB78E4C5
:101D23007930121E0C753490753501753600753790
:101D330000120648783879E0121E0C121DB378ECB5
:101D43007930121E0CE53075F003A4F53078307944
:101D5300E0121E0C121DB378EC7930121E0CE53024
:101D630075F002A40475F00584F530783079E0123B
:101D73001E0C121DCB78E87930121E0C78DC7934F6
:101D8300121E0C1205C7783879DC121E0C78DC752C
:101D9300F001121DE378DC7930121E0C75340775DF
:101DA3003500753600753700120648E53CF56022AC
:101DB30078DC7930121E0C78E07934121E0C12058F
:101DC300C7783879DC021E0C78DC7930121E0C7867
:101DD300E07934121E0C1205DF783879DC021E0C10
:101DE300E625F0F608E63400F608E63400F608E6E1
:101DF3003400F622C3E695F0F608E69400F608E60A
:101E03009400F608E69400F622E6F70809E6F708D8
:101E130009E6F70809E6F722C0E023232323540F3A
:101E2300F5F0D0E0540F227549007548007547005E
:101E3300754600754500754400754300754200758D
:101E4300410075400022E579B40109207A0122C2DC
:101E53007A021F96E55F455E455DB4000122E55FAA
:101E6300121FC5F55FB49917755F99E55E121FC51B
:101E7300F55EB4990A755E99E55D121FC5F55D00BF
:101E8300E55F455E455DB40002800122121F9602A4
:101E93001E95C082C083C0F088F0C0F07800121F86
:101EA30064120C83B4FF02804EB55B3DA3120C8316
:101EB300B4005C121F64A3A3E560B406028007B4F8
:101EC300000280028003A3A3A3120C83F55DA31277
:101ED3000C83F55EA3120C83F55FE55D455EB400EC
:101EE3000B855F78755F0080030880B2D0F0A8F09F
:101EF300D0F0D083D08222122D54901F061202A656
:101F0300022EA74272616B207461727966790012A6
:101F13001F64120C83F507A3120C83F5F0E563B578
:101F2300F0005011121F5A120C83B5070280F512EC
:101F33001F5F021EB6121F5A120C83B507F1A312BC
:101F43000C83F5F0E563B5F00050EA80E2755D00BF
:101F5300755E00755F002208E8021F6418E8021F1F
:101F6300648882758300E58233F582E58333F583E4
:101F7300E58233F582E58333F583E5823354F8F55F
:101F830082E58333F583E5822410F582E58334000B
:101F9300F58322E5782401D4F578E5773400D4F588
:101FA3007722757801757700C27A22757800757784
:101FB3000075190075180022757600757500757423
:101FC3000022B40003749922C39401C0E0540FB4F7
:101FD3000F07D0E054F0440922D0E022121334C09A
:101FE300508510501203031214279020081202A6E2
:101FF30012208F12216F1221541220F8122B3C123F
:102003003365D050220D0A4B6F6E66696775726136
:10201300636A613A0D0A20202053706F73056220B2
:1020230020202020202043656E6120202020547929
:1020330070202020202020537464616E64617264D8
:10204300504C20537464616E64617264504C0D0A89
:102053002020207A616C69637A616E696120202097
:10206300696D70756C7375204472756B61726B6901
:10207300204472756B61726B692020202052532DAE
:10208300323332430D0AFB392D0D0A00740312213A
:1020930049E579B400069020C40202A6B401069073
:1020A30020D10202A6B402069020DE0202A6C0E0FE
:1020B3009020EC1202A6D0E01201AC9020F00202B4
:1020C300A6506F6C6172797A61636A612000496D11
:1020D30070756C732031366B487A005A616E696B88
:1020E30020343030487A202000506F200020736560
:1020F3006B2E2020007406122149E5111221097468
:1021030003122149E51290213FB40103902121B428
:10211300020390212BB403039021350202A6416DE3
:10212300696761504C20200057696E646F77735064
:102133004C004D617A6F776961504C0042657A506B
:102143004C2020202000C0E01202E5D0E0D5E0F6CC
:10215300227403122149E50F902167B402039021F1
:102163006B0202A650617200536572001202E5E52C
:10217300591201AC742C120704E55A1201AC22D295
:102183006C8002C26C121334C0508510501221E0CF
:10219300D050E510B4030312219E2212016790214F
:1021A300B51202A612132520D5055003121162029F
:1021B30003030C4B61736F776102206275666F7264
:1021C300203F000C496E6974206B6F6E666967204F
:1021D3003F000C4E617065776E6F203F0012030362
:1021E3001214279023671202A6757B00757C0120C9
:1021F3006C0E121211500C9023DF1202A6022361FF
:10220300120D67306C0B120C47547FB47F0B022303
:1022130017120C47500302231FC0E0751500122A42
:10222300ACC083C082857C82857B8375F0041217E2
:1022330064D082D083D0E01202E51201AC742F1275
:102243000704120C471201AC1202E5120C471201EB
:10225300AC743A120704120C471201AC1202E57F68
:102263000678F0120C4712262FC0E0030303035431
:102273000FF608D0E0540FF608DFE8C083C08212DF
:1022830014E0855C827583001215261202E5E5676A
:102293001201AC1202E51213AED082D0831202E512
:1022A300120C471201AC743A120704120C471201C4
:1022B300AC742E120704120C471201AC1202E51281
:1022C3000C47FD7F007E00120C47FCC083C0828D4B
:1022D300838C8275F0041217641202E575F00A12FA
:1022E30023F5AF15120C47B5070280069023EE12B3
:1022F30002A6D082D083E57C2401D4F57CE57B342F
:1023030000F57B120303120EEC4011206C06120D34
:102313006F022206120D6F4003022206206C3F90CB
:1023230023D31202A61211CC121E2AEF121E1B85F2
:10233300F047F546EE121E1B85F045F544ED121EDF
:102343001B85F043F542EC121E1B85F041F54075E9
:10235300F0081217961202E575F00A1223F512031C
:1023630003022B3C0D0A57796472756B2064616E0E
:102373007963682072656A6573747261746F7261E0
:102383000D0A0D0A4C702E202044617461202047F1
:102393006F647A20204E722074656C65666F6E756B
:1023A300205461722053747265666120202020439B
:1023B3007A617320202020204C69637A6E696B2038
:1023C3002020202043656E610D0AFB442D0D0A0079
:1023D3000D0AFB2A2053756D613A20000D0A4275E0
:1023E300666F722070757374792100202D204572F9
:1023F3007200C0F0EF121E2A121E1B85F047F5462D
:10240300EE121E1B85F045F544ED121E1B85F043AD
:10241300F542EC121E1B85F041F540120473853B17
:1024230033853A32853931853830122481120604D6
:102433001204AFD0F012243C22C2D130F702D2D121
:10244300E5F0543FF5F0743F25F0F8D2D5E630D5EA
:10245300196004C2D58013E5F0B40306C2D5743005
:10246300800820D1081202E58003120201E8C39418
:1024730040B40205742C12070418D5F0D022E55994
:10248300121E1B121E2A85F043F542E55A121E1B2B
:1024930085F041F540120473853B37853A3685391B
:1024A3003585383422C0E0E55725F0F557E5563435
:1024B30000F556D0E022121334C050851050120399
:1024C300031214279025461202A61224D9122B3C7C
:1024D300123365D050227800120EEC4065121F644F
:1024E300120C83B4FF02805AC0E07474120704D044
:1024F300E01201AC1202E5A3120C831201AC7403C7
:10250300122149A3120C83120201A3120C8312019C
:10251300AC742C120704A3120C831201AC740412C2
:102523002149A3120C83120201A3120C831201ACE2
:10253300742C120704A3120C831201AC12030308B8
:102543008096220D0A2338330D0A54617279667915
:102553000D0A4E7220476F647A20446E6920706FB3
:1025630077737A20446E692006776908740D0AFB35
:102573001D2D0D0A00121334C05085105012030391
:102583001214279025F81202A6122598122B3C123A
:102593003365D050227A00120EEC40121225B2405D
:1025A3000D1202E5A31213B11203030A80E92212EA
:1025B3001583120C83B4FF02D322C0E07470120798
:1025C30004A3120C8312262FA3120C8312262FA30B
:1025D300120C8312262FA3120C8312262FA3120C84
:1025E3008312262FA3120C8312262F1202E5D0E0AA
:1025F3001201ACC3220D0A2338320D0A50726566EC
:10260300696B73790D0A2020204E72202020202030
:1026130020202020546172204F7069730D0AFB152E
:102623002D0D0A00C0E0C082C0838017C0E0C082C5
:10263300C083C0E003030303540F9026569312078D
:1026430004D0E0540F90265693120704D083D0820F
:10265300D0E02230313233343536373839412A230A
:1026630044455FC0E0C082C083C0E003030303545A
:102673000F90268D93120704D0E0540F90268D936C
:10268300120704D083D082D0E02230313233343584
:1026930036373839412A23444520C083C082C0F0ED
:1026A300C000F5F09026E5780DE493B5F007122607
:1026B300C6E4938005A3D8F1E5F0D000D0F0D08232
:1026C300D08322780DE551B40102781AB40202785E
:1026D30027B403027834E58228F582E5833400F5D4
:1026E300832208010203040506070A0D0CFDFC61A1
:1026F30065636C6E6F737A0A0D0D0D0CE2EBEAEEF7
:10270300EFF3F4FB0A0D0A0A0CB9EAE6B3F1F39C02
:10271300BF0A0D0D0D0C86918D92A4A29EA70A0DE2
:102723000D0D0CC083C082C0F0C000C007F5F0E5FA
:1027330051B40002801A9026E51226C6780D7F0058
:10274300E493B5F007EF9026E5938006A30FD8F046
:10275300E5F0D007D000D0F0D082D08322C0D0C023
:10276300E0C0F0C000C001C002C003C004C005C087
:1027730006C007C083C082209925E599C298122715
:10278300EA122EE8D082D083D007D006D005D00439
:10279300D003D002D001D000D0F0D0E0D0D032D2DC
:1027A30077C29980DCC0F0C000E555B40025C2AC07
:1027B300E554B40008C3D2ACD000D0F0221554A81D
:1027C30052E6C0E00552E552B4DB037552C0D0E0D7
:1027D300D380E3755001122D549027E51202A6020F
:1027E3002EA74649464F00A853F60553E553B4DBDD
:1027F300037553C00554E554B41B05755501D32225
:10280300C3227554007555007553C07552C022C25A
:102813007AD288D2A8C28922C27BD28AD2AAC28B98
:102823002275985043878053890F438920758DCB38
:10283300758BCBD28ED277D2AC22757E0A122EE85C
:102843001227A84006E57E70F4D322122726C3225E
:102853001227A850FB80F4C0F012283D4014122820
:1028630079C4F5F012283D400912287945F0D0F0DB
:10287300C322D0F0D322B42003740022B45F0374C4
:102883000F22B460005009B440005008C3943022B2
:10289300C3945722C3943722C0E01228A6D5E0FA86
:1028A300D0E022C0E0740A1228C4D5E0FAD0E022B6
:1028B300C0E074051228C4D5E0FAD0E0220228C48F
:1028C30022C26B122EE8306BFD22C0E01228D8D54D
:1028D300E0FAD0E022C0E074F7D5E0FD74F7D5E06C
:1028E300FDD0E022751500900000120C83122AAC73
:1028F300900001120C83F579122AAC900002120C9D
:1029030083F55A122AAC900003120C83F559122A4C
:10291300AC900004120C83F558122AAC90000512F7
:102923000C83F513122AAC900006120C83F51412D3
:102933002AAC900007120C83F512122AAC900008FF
:10294300120C83F511122AAC900009120C83F50FB7
:10295300122AAC90000A120C83F529122AAC9000BB
:102963000B120C83B5150A900000120C83B40306F6
:1029730022740102297E740802297E4517F5172265
:10298300744012017EE517B4000122D28213500570
:102993009029C880291350059029D9802113500507
:1029A3009029E880191350059029F98011135005D7
:1029B300902A0A8009135005902A168001221202D8
:1029C300A61228A6225A03612073756D61206B6FCE
:1029D3006E66696775005A03612073756D612074B3
:1029E30061727966005A03612073756D612070729C
:1029F3006566696B73005A036120776572736A6158
:102A0300206B6F6E662E004275666F7220706503D1
:102A13006E79005A6F737461036F20313025206221
:102A230075662E007515009000007403120CDC12FD
:102A33002AAC900001E579120CDC122AAC9000025A
:102A4300E55A120CDC122AAC900003E559120CDC97
:102A5300122AAC900004E558120CDC122AAC900048
:102A630005E513120CDC122AAC900006E514120CD7
:102A7300DC122AAC900007E512120CDC122AAC908F
:102A83000008E511120CDC122AAC900009E50F12C4
:102A93000CDC122AAC90000AE529120CDC122AACD9
:102AA30090000BE515120CDC222515F51522122DCD
:102AB30054902ABA0202A6437A61730D0A001203E4
:102AC30003122D54902ACD0202A6536B0361646E48
:102AD30069610D0A00E554B40004755001221228FF
:102AE3003DB423F1C29575500275100212133412CE
:102AF300030312030312285A40B412107150DBB4BB
:102B0300820F122C85122DC6122B57122C63022A08
:102B1300DDB4830F122BC5122DC7122B8E122C631B
:102B2300022ADD122AC17550021203037900120E24
:102B33006740030980F8022ADD902B481202A6128F
:102B4300015D02018F0D0A0D0A4B6F6E6965630DFE
:102B53000A0D0A00122B62E515120CDC0207AA7596
:102B630015007A00121583120C83A3B4FF0C120C08
:102B730083B5150122740402297E122AAC7F0F1239
:102B83000C83A3122AACDFF70A80D9122B99E5151F
:102B9300120CDC0207AA7515007800121F64120CD0
:102BA30083A3B4FF0C120C83B5150122740202290E
:102BB3007E122AAC7F07120C83A3122AACDFF7081C
:102BC30080D9902D7F1202A67800122DA650030201
:102BD3002C70B44B08121F6474FF020CDCB474EA4B
:102BE300E8B43103022C73E8122D37121F64122844
:102BF3005A120CDCA312283DB4205F12285A120C7F
:102C0300DCA312283DB4205212283DB4204C1228D4
:102C13005A120CDCA312285A120CDCA312283DB45E
:102C23002C3812285A120CDCA312283DB4202B1284
:102C3300283DB4202512283DB4201F12285A120C17
:102C4300DCA312285A120CDCA312283DB42C0B125D
:102C5300285A120CDCA308022BCD122AC1022D2CF8
:102C6300902C690202A60D0A4F4B0D0A00022AB1ED
:102C7300122D64121F6474FF120CDC12283DB44B36
:102C8300FA22902D7F1202A67A00122DA640DEB4FE
:102C93004B0812158374FF020CDCB470EDEAB4C761
:102CA30003022D29EA122D3712158312285AFF1217
:102CB300285AFE12285AFD12285AFC12285AFB12CF
:102CC300285AF912283DB4205812285A120CDCA3B2
:102CD300EF120CDCA3EE120CDCA3ED120CDCA3EC64
:102CE300120CDCA3EB120CDCA3E9120CDCA31228FC
:102CF3003DB4202D790912283DB40D028003B40A96
:102D0300077400120CDC800A120CDCA3D9E80A0257
:102D13002C8D7400120CDCA3D9F8122DB30A022CEB
:102D230092122AC18003122D6412158374FF120CB0
:102D3300DC022C7EC0F0C0E0740D120704D0E01258
:102D43000317C0E0E5F0120201D0E01201ACD0F0AD
:102D530022D282902D5C0202A60C420308643A2020
:102D630000122D54902D6D0202A6440375676F0661
:102D730002207461626C6963790D0A000D0A57635E
:102D83007A7974756A01207461626C6963012E2E0D
:102D93000D0A00902D9C0202A60C536F7274756A83
:102DA30001200012283D4019B40D028003B40AF338
:102DB30012283D400CB40D0280F6B40A0280F1C320
:102DC30022D32222122DFDE5F0602E7900122D96DA
:102DD300EE1201AC742F120704E5F01201AC780077
:102DE300C26D122E135005122E50D26D08E8B5F0A5
:102DF300F1306D050EEEB5F0D4227800121F641287
:102E03000C83B4FF0280030880F21888F07E00224E
:102E1300C000C0F0122E8008121F6479F1E7F5F0AC
:102E2300A3120C83C395F0C0D019E7F5F0122E3F1F
:102E3300120C83D0D095F0D0F0D00022C0E01582E0
:102E4300E582B4FF051583D0E022D0E022C0001252
:102E53002E8008121F647F0779F0120C83C0E0E70D
:102E6300120CDCD0E0F709A3DFF018121F647F0710
:102E730079F0E7120CDC09A3DFF8D00022121F64FB
:102E83007F0879F0120C83F709A3DFF822122D547F
:102E9300902E9C1202A6022EA757790308637A6F1D
:102EA3006E652100120167C2AF741E122EC2122E6C
:102EB300E8D5E0F7741E122EC2D5E0FA0200007FB7
:102EC3000A7E64120101DEFBDFF922C276C2A9C2C7
:102ED300A81203AA74401203D24002D2761203C28C
:102EE300D2A9D2A822C0E0B29400B294D0E02222A8
:102EF300C26D122FCA7A0012018F12015D1225B220
:102F030040F3120303A31213B1120F0B20D5744025
:102F1300F8B40007D26D122F8980DAB401030A8056
:102F2300D6B402091AEAB4FFCEAAF080CAB4030DDC
:102F330012310FFAB5F00040BEAAF080BAB404070C
:102F4300D26D122FEE80B0B4051FD26D05F0E5F0FF
:102F5300B4C70050A0AAF0122FEEC0020A121583C4
:102F630074FF120CDCD002808EB4070EC002C0F0D6
:102F7300122578D0F0D002022EFAB4098C306D03FA
:102F8300122DC6022B57902FA71202A6EAB5F00204
:102F93008008122FB10AEAB5F0F8AAF0121583746B
:102FA300FF020CDC0C4B6173756A012E2E00C0020C
:102FB3000A122FDE1A1215837F1078F0E6120CDC4A
:102FC30008A3DFF8D002227A00121583120C83B40F
:102FD300FF0280030A80F21A8AF0221215837F10FF
:102FE30078F0120C83F608A3DFF822120167903001
:102FF3006C1202A6121583A3757F407E06120E8BF8
:1030030020D565B4CC0A74FF120CDCA3DEF880185B
:10301300FD540FB40C0BED440F120CDCA3DEE78060
:1030230007ED120CDCA3DED590307E1202A612153A
:1030330083757F07120E8B20D52E120CDC90308601
:103043001202A6121583A3A3A3A3A3A3A3757F4070
:103053007E0912309120D510B4CC077400120CDC19
:103063008006120CDCA3DEEA220C5770726F7761C4
:1030730064072070726566696B73000C5461727922
:103083006661000C4B6F6D656E7461727A00C0836C
:10309300C082C0F0120E9D20D520B4CC02801BF557
:1030A300F09030C4E493B4FF0280E9B5F008A3E4E0
:1030B300931207048004A3A380EAD0F0D082D083C4
:1030C300220B200030103120323033403450356031
:1030D30036703780389039214122422343314432BC
:1030E300453346414742484349514A524B534C6149
:1030F3004D624E634F7150725273538154825583A4
:10310300569157925893590251035AFF12016790EF
:1031130031251202A6757F0B120E8B20D5031231B7
:1031230031220C4E722072656B6F72647500C0F0B1
:10313300C007C00675F000FFC4540F600AFEC3E564
:10314300F0340AF5F0DEF8EF540F25F0D0F0D00696
:10315300D00722C26D122DFD780012018F12015D7E
:103163001231E440F3120F0B20D57340F8B400077B
:10317300D26D1232D680E3B401030880DDB40209B4
:1031830018E8B4FFD5A8F080D1B4030D12310FF8BD
:10319300B5F00040C5A8F080C1B40407D26D123267
:1031A3002480B7B4051FD26D05F0E5F0B4310050AB
:1031B300A7A8F0123224C00008121F6474FF120C77
:1031C300DCD0008095B4070DC000C0F01224B9D044
:1031D300F0D0008085B4098D306D03122DC7022B0A
:1031E3008E121F64120C83B4FF02D322C0E07474E6
:1031F300120704D0E01201AC1202E5A3120C8312F1
:1032030001AC1202E5A3120C83120201A3120C8378
:103213001201AC742C120704A3120C831201ACC369
:10322300221201679032A11202A6121F64757F4019
:10323300120E8B20D567120CDCA3757F44120E8B04
:1032430020D55A120CDCA3757F49120E8F20D54D61
:10325300120CDCA3120E8B20D543120CDC742C123F
:103263000704A3120E8B20D534120CDCC083C0825A
:103273009032B11202A6D082D083A3120E8F20D532
:103283001C120CDCA3120E8B20D512120CDC742C36
:10329300120704A3120E8B20D503120CDC220C544C
:1032A300617220476F647A204F6B726573000C570D
:1032B3006F6C6E6520646E692000C00008122E805A
:1032C30018121F647F0879F0E7120CDC09A3DFF8FA
:1032D300D00022902FA71202A6E8B5F002800812B0
:1032E30032BD08E8B5F0F8A8F0121F6474FF020CB1
:1032F300DC1201679033171202A6120E8B20D5132E
:10330300F5F0120E8B20D50BB51407E5F0B51302BB
:10331300C322D3220C4B6F64200012016790331732
:103323001202A6120E8B20D52DFF120E8B20D5264E
:10333300FE90335A1202A6120E8B20D519FD120EDF
:103343008B20D5128EF0B5F0D1EF8DF0B5F0CB8F89
:10335300138E14122A27220C506F6E6F776E6965D5
:103363002000E550B403069033711202A6220D0A21
:10337300FC001211CCEAB52709EBB528057410023D
:10338300297E85278285288375F003E58303F583EA
:10339300E58213F582D5F0F3C3E5279582FCE52892
:1033A3009583FDC3EA9CEB9D4005742002297E2290
:1033B300120D5912018F120D8F120C47500B902BC7
:1033C3004C1202A6741402289B1201AC742F12072C
:1033D30004120C471201AC1202E5120C471201ACA5
:1033E300743A120704120C471201AC1202E51203DD
:1033F300037F04120C4712262FDFF87F02120C47BB
:1034030054F0B4F00474208002743EF5F0DF0280BF
:1034130005120C47DFFB120C47120C47120C47E551
:10342300F01207041202E5120C47FD120C47FC7F51
:10343300007E0075F0051223F53092FD75F032120F
:1034430028A62092030233B6D5F0F42212018F7816
:1034530000E81234705009E81201AC74201207041A
:1034630018D8EE7465120704122EE880FB1203AA23
:103473001203D240051203C2D3221203C2C3221283
:1034830001679021C61202A612132520D50240011E
:10349300229021D51202A612132520D5F340012232
:1034A30090352B1202A6757900755900755A35753A
:1034B3005822751100751200750F017513117514DB
:1034C30011122A277A00121583AC82AD839036201D
:1034D300AE82AF838E828F83E493A3AE82AF838C5D
:1034E300828D83120CDCA3AC82AD83BEA1E6BF3612
:1034F300E3122B577800121F64AC82AD83903539E9
:10350300AE82AF838E828F83E493A3AE82AF838C2C
:10351300828D83120CDCA3AC82AD83BE1AE6BF3668
:10352300E3122B8E122C63220C496E69742E2E002B
:1035330053746454617200000B00000B000001001F
:103543000C00000C0000020801800003600002224E
:1035530003600003600003000060000060000408D3
:10356300004350005800041800870000870006003D
:1035730000311000311007000008700008700800C7
:1035830000043600043609080012400016600918CA
:103593000016600016600922002490002490100099
:1035A30000125000125011000011200011201200CF
:1035B30000103000103013000009320009321400EB
:1035C300000830000830150000050400050416004B
:1035D30000028000028017080180000360001718B2
:1035E30003600003600019080043500058001918D5
:1035F300008700008700200800435000580020186F
:10360300008700008700210800435000580021185C
:10361300008700008700FF53746450726502FFFF48
:10362300FFFFFFFF4C6F6B616C6E6120200099FF01
:10363300FFFFFFFF416C61726D6F77792009050110
:10364300FFFFFFFF49646561202020202009060F4A
:10365300FFFFFFFF47534D20202020202009069223
:10366300FFFFFFFF47534D20202020202009090F93
:10367300FFFFFFFF43656E74657274656C040FFF93
:10368300FFFFFFFF4D2F4D2020202020201600FF9D
:0E369300FFFFFFFF5A616772616E696361FF9E
:00000001ff
